:0300330002002D9B
:04002D0053D8EF3283
:10004600300918121333EFC3953C40030200D890D1
:100056007FBF7401F0C209C200807730033B907FF6
:10006600C6E020E16D121333EFC394405064907ED6
:1000760040E0139209907FC7E014F5192000116043
:100086000FF5087E7E7F41750C7E750D41120CCCF6
:10009600C203E4907FC7F08039907FC8E020E13248
:1000A600121333EFC394405029907DC0E013920998
:1000B600907FC9E014F519200011600FF5087E7DC8
:1000C6007FC1750C7D750DC1120CCCD203E4907FF7
:1000D600C9F0907FB6E030E1030201601211F58F9E
:1000E6001912133F8F36E519C3953A500F12131B99
:1000F600EF30E008E53620E703300B5EC20BE5196A
:0C003600907F987410F090C000E0FF2252
:03004300021300A5
:10000300C0E0C083C082C085C084C086758600906E
:100013007FC4E4F05391EF907FAB7404F0D086D0AB
:0A00230084D085D082D083D0E03273
:03000000020E12DB
:400106006058B48003433602E53630E726E519D3942040037519208519087E7E7F80750C7E750D80AF36120F5DE51925E0907FB7F08027E519D3943F400375193F851908C2
:40014600907E80E536F07E7E7F81750C7E750D81120CF1E51904907FB7F0907FCEE030E1062005030203C1E4F51874402518F582E4347CF583E0FFE5187C007B017A7E79AF
:40018600002400F9EC347EFAEF120EE40518E518B420D7907E00E06068907E03E060247F01E4FD1211D07F037DCD1211D0434680907F987414F090C000E546F0E4907E13F6
:4001C600F08030907E01E0FF121054907E02E0FF12107A7F01907E11E0FD1211D07F037D071211D0434680907F987414F090C000E546F0907F987412F0E540440690C00093
:40020600F0907E03E07006907E13E07008E4907E13F07525FF907E05E06012A3E0543FF544907F987413F090C000E544F0907E07E0602BA3E06005434280800353427F53C8
:4002460042FC907E09E06011434202A3E0FF1210C6907E0BE0FF1210ECAF421210A0907E03E0600853427FAF421210A0907E0CE06018A3E0600543460280035346FD907FFB
:40028600987414F090C000E546F0907E0EE06018A3E0600543460180035346FE907F987414F090C000E546F0907E12E0F53AA3E013920DA3E0F53CA3E06005434610800317
:4002C6005346EF907F987414F090C000E546F0907E16E060325344BF907F987413F0E544547F90C000F0907F987411F012130FEF54FE90C000F0533EFDE4FFAD3E1211D080
:40030600E4F52AF529D207907E17E0600F433E02E4FFAD3E1211D0752901D207907E18E06010907F987412F0E540440490C000F0D200907E19E06011434440907F9874130E
:40034600F0E544547F90C000F0907E1AE0600F533EFEE4FFAD3E1211D0752B01D207907E1BE0600F433E01E4FFAD3E1211D0E4F52BD207907E1CE0600E907F987412F0E5F8
:4003860040440290C000F0907E1DE06002D20B907E1EE06008752C01E4F538D207907E1FE06011907FD77411F07431F07415F07435F0D203C205E4907FCFF0301A54E5389E
:4003C6006002153820134BE513D3940040041513804075130A301B02D21312130FEF5401F519652A600585192AD20712134BEF54806480F51965266005851926D207300D71
:400406001112134BEF5410F51965256005851925D207201B030207F0300A18121387EFC3953D40030204B0907FC17401F0C20AC200807730043B907FCAE020E16D1213879B
:40044600EFC394405064907D40E013920A907FCBE014F519200011600FF5087E7D7F41750C7D750D41120D16C204E4907FCBF08039907FCCE020E132121387EFC394405099
:4004860029907CC0E013920A907FCDE014F519200011600FF5087E7C7FC1750C7C750DC1120D16D204E4907FCDF0907FBAE030E10302053812123F8F191213938F37E5197F
:4004C600C3953B500F12136FEF30E008E53720E703300C5EC20CE5196058B48003433702E53730E726E519D3942040037519208519087E7D7F80750C7D750D80AF37120FFC
:4005060096E51925E0907FBBF08027E519D3943F400375193F851908907D80E537F07E7D7F81750C7D750D81120D3BE51904907FBBF0907FD0E030E106200603020799E431
:40054600F51874C02518F582E4347BF583E0FFE5187C007B017A7E79202420F9EC347EFAEF120EE40518E518B420D7907E20E06068907E23E060247F01E4FD12121A7F03F7
:400586007DCD12121A434780907F98740CF090C000E547F0E4907E33F08030907E21E0FF121138907E22E0FF12115E7F01907E31E0FD12121A7F037D0712121A43478090AA
:4005C6007F98740CF090C000E547F0907F98740AF0E541440690C000F0907E23E07006907E33E07008E4907E33F0752EFF907E25E06012A3E0543FF545907F98740BF090EB
:40060600C000E545F0907E27E0602BA3E06005434380800353437F5343FC907E29E06011434302A3E0FF121184907E2BE0FF1211AAAF43121112907E23E0600853437FAFA0
:4006460043121112907E2CE06018A3E0600543470280035347FD907F98740CF090C000E547F0907E2EE06018A3E0600543470180035347FE907F98740CF090C000E547F0B4
:40068600907E32E0F53BA3E013920EA3E0F53DA3E0600543471080035347EF907F98740CF090C000E547F0907E36E060325345BF907F98740BF0E545547F90C000F0907F79
:4006C600987409F0121363EF54FE90C000F0533FFDE4FFAD3F12121AE4F533F532D208907E37E0600F433F02E4FFAD3F12121A753201D208907E38E06010907F98740AF0EB
:40070600E541440490C000F0D200907E39E06011434540907F98740BF0E545547F90C000F0907E3AE0600F533FFEE4FFAD3F12121A753401D208907E3BE0600F433F01E4C9
:40074600FFAD3F12121AE4F534D208907E3CE0600E907F98740AF0E541440290C000F0907E3DE06002D20C907E3EE06008753501E4F539D208907E3FE06011907FD7741369
:40078600F07433F07416F07436F0D204C206E4907FD1F0301A54E5396002153930134BE513D3940040041513804075130A301B02C213121363EF5401F51965336005851998
:4007C60033D20812139FEF54806480F519652F600585192FD208300E1112139FEF5410F519652E600585192ED208301A2A907FD2E020E123907B40E06009E0F515907B4297
:40080600E0F516907B41E06009907FD77417F07437F0E4907FD3F0907FC2E030E103020924E50A7040300739E5387035C207F5187E007B0074242518F9EE3400FA120E9E44
:40084600FF74802518F582E4347BF583EFF00518E518B409DB907FC37409F0753810E4F52C750A0122E50A64017040300839E5397035C208F5187E007B00742D2518F9EEBF
:400886003400FA120E9EFF74802518F582E4347BF583EFF00518E518B409DB907FC37409F0753910E4F535750A0222E50A6402703630142FC214F5187E007B00740E25184C
:4008C600F9EE3400FA120E9EFF74802518F582E4347BF583EFF00518E518B405DB907FC37405F0750A0322E51560301515E4F5187E007B0074142518F9EE3400FA120E9ECB
:40090600FF74802518F582E4347BF583EFF00518E518B403DB907FC37403F0E4F50A22907FE9E0120EF60A0C000A80010AEC0309480609FF0809F90909E10A09F00B000044
:400946000B3B907FEBE024FE6019146061240260030209D77419907FD4F07400907FD5F0020B42907FEAE070047F0280027F03758282758319EFF075827B758319F07582DA
:4009860074758319F0758266758319F0758258758319F0907FEAE004758217758319F07419907FD4F07412907FD5F0020B42907FEAE0FF120F1CEA49600DEA907FD4F0E9BE
:4009C600907FD5F0020B42907FB4E04401F0020B42907FB4E04401F0020B42907F00E509F0907FB57401F0020B42907FEAE0F509020B42120B4A020B42907F007401F0903B
:400A06007FB5F0020B42907FE8E0247F60241460312402705BA210E433FF25E0FFA216E4334F907F00F0E4A3F0907FB57402F0020B42E4907F00F0A3F0907FB57402F0022E
:400A46000B42907FECE0F45480FFC4540FFFE054072F25E024B4F582E4347FF583E054FD907F00F0E4A3F0907FB57402F0020B42907FB4E04401F0020B42907FE8E024FE4E
:400A8600601D24026003020B42907FEAE0B40105C210020B42907FB4E04401F0020B42907FEAE07038907FECE0F45480FFC4540FFFE054072F25E024B4F582E4347FF583EA
:400AC600E4F0907FECE05480FF131313541FFFE054072F907FD7F0E04420F0805F907FB4E04401F08056907FE8E024FE60182402704A907FEAE0B40104D210803F907FB47B
:400B0600E04401F08036907FEAE07020907FECE0F45480FFC4540FFFE054072F25E024B4F582E4347FF5837401F08010907FB4E04401F08007907FB4E04401F0907FB4E017
:400B46004402F022E4907F93F0907F9C7430F0E4907F96F0907F9574C0F0907F9E743FF0907F987418F0E4F58E907FDF74FFF0907FDEF0E4F5247518017B0074242518F945
:400B8600E43400FAE4120EE40518E518B409EA753A01E4F538F513F536C207C20BC205C200C209C213907F987413F075440390C0007403F07F0CE4FD1211D07F108F42125F
:400BC60010A0907F987412F07F018F40EF440690C000F0907F987414F075468090C0007480F00FE4FD1211D0E4FF7EA3AD068D3E1211D0907F987411F090C000E4F07F05B0
:400C06007D7F1211D07F011212897F037D071211D07F137D091211D0201B03020CC9752D017518017B00742D2518F9E43400FAE4120EE40518E518B409EA753B01E4F53978
:400C4600F513F537C208C20CC206C200C20AC213907F98740BF075450390C0007403F07F0CE4FD12121A7F108F43121112907F98740AF07F018F41EF440690C000F0907FC0
:400C860098740CF075478090C0007480F00FE4FD12121AE4FF7EA3AD068D3F12121A907F987409F090C000E4F07F057D7F12121A7F011212AA7F037D0712121A7F137D0927
:400CC60012121AD21222907F987410F0AF08E50DF582E50CF583C2AF058690C0000586E0A30586F00586DFF7D2AF22907F987410F0AF08E50DF582E50CF583C2AF058690FD
:400D0600C000E00586F0A30586DFF70586D2AF22907F987408F0AF08E50DF582E50CF583C2AF058690C0000586E0A30586F00586DFF7D2AF22907F987408F0AF08E50DF53A
:400D460082E50CF583C2AF058690C000E00586F0A30586DFF70586D2AF227400F58690FDA57C05A3E582458370F922907FD6E04480F0438701000000000022D219907F92B8
:400D8600E04402F0907FAEE0FFD39210E433FEEF4EF0D2E843D820907FDE7401F0907FDFF0907FAB74FFF0907FA9F0907FAAF05391EF907FAFE04401F0907FAEE0440DF0AD
:400DC600D2AFD21A121264C211E4F50BF513C217C212907FA104F0907FD8E065176010301205D21A120046907FD8E0F5178008301205C21A120046301107C21112092580F9
:400E0600D63018D3C2181213AB80CC22787FE4F6D8FD758147020E59020D81E493A3F8E493A34003F68001F208DFF48029E493A3F85407240CC8C333C4540F4420C88340FA
:400E460004F456800146F6DFE4800B01020408102040809012CBE47E019360BCA3FF543F30E509541FFEE493A360010ECF54C025E060A840B8E493A3FAE493A3F8E493A320
:400E8600C8C582C8CAC583CAF0A3C8C582C8CAC583CADFE9DEE780BEBB010689828A83E0225002E722BBFE02E32289828A83E49322BB010CE58229F582E5833AF583E022D5
:400EC6005006E92582F8E622BBFE06E92582F8E222E58229F582E5833AF583E49322BB010689828A83F0225002F722BBFE01F322D083D082F8E4937012740193700DA3A37A
:400F060093F8740193F5828883E4737402936860EFA3A3A380DF8F18E4F519751AFF751B19751C86AB1AAA1BA91C900001120EB7B4031DAF190519EFB5180122120E9E7EC4
:400F46000029FFEE3AA907751AFFF51B891C80D47B007A007900228F1A050DE50DAE0C7002050C14F5828E83E51AF0120036050DE50DAC0C7002050C14F5828C83EFF015BA
:400F860008E508600A12133F8F1AEF423680CA228F1A050DE50DAE0C7002050C14F5828E83E51AF0121357050DE50DAC0C7002050C14F5828C83EFF01508E508600A1213AA
:400FC600938F1AEF423780CA22E4907F93F0907F9C7430F0E4907F96F0907F95F0907F9E7427F0907F987420F0907F9E7407F0E4907F94F0907F9D74FFF0E4907F97F0227C
:40100600C0E0C083C082C085C084C086758600D2115391EF907FAB7401F0D086D084D085D082D083D0E032C0E0C083C082C085C084C086758600D2185391EF907FAB74087E
:40104600F0D086D084D085D082D083D0E032907F987413F090C00074BFF0907F987410F090C000EFF0907F987413F0E544547F90C000F022907F987413F090C00074BFF00C
:40108600907F987411F090C000EFF0907F987413F0E544547F90C000F022907F987413F090C00074BFF0907F987412F090C000EFF0907F987413F0E544547F90C000F0220A
:4010C600907F987413F090C00074BFF0907F987414F090C000EFF0907F987413F0E544547F90C000F022907F987413F090C00074BFF0907F987416F090C000EFF0907F9807
:401106007413F0E544547F90C000F022907F98740BF090C00074BFF0907F98740AF090C000EFF0907F98740BF0E545547F90C000F022907F98740BF090C00074BFF0907FFA
:40114600987408F090C000EFF0907F98740BF0E545547F90C000F022907F98740BF090C00074BFF0907F987409F090C000EFF0907F98740BF0E545547F90C000F022907F71
:4011860098740BF090C00074BFF0907F98740CF090C000EFF0907F98740BF0E545547F90C000F022907F98740BF090C00074BFF0907F98740EF090C000EFF0907F98740BFD
:4011C600F0E545547F90C000F022907F987413F0E544547F90C000F0907F987417F090C000EFF0907F987415F090C000EDF0221213278F1A1213278F1BE51A651B60121292
:4012060013278F1AE51A651B60071213278F1B80E8AF1A22907F98740BF0E545547F90C000F0907F98740FF090C000EFF0907F98740DF090C000EDF02212137B8F1A121325
:401246007B8F1BE51A651B601212137B8F1AE51A651B600712137B8F1B80E8AF1A22907FD6E054FBF0E04408F0301A04E04402F07FF47E011212E7907FD6E054F7F0E044E1
:4012860004F022AE07E4FFE53E547FFD1211D0907F987411F090C000EEF0E4E53E4480FD1211D022AE07E4FFE53F547FFD12121A907F987409F090C000EEF0E4E53F448095
:4012C600FD12121A22050E02000000000314030000C111C118C195C110C116010A00C19B008E188F19E5191519AE18700215184E6005120D6080EE2200000210060002137E
:4013060004000200030002102D907F987411F090C000E0FF22907F987412F090C000E0FF22907F987413F090C000E0FF22907F987414F090C000E0FF22907F987415F090F5
:40134600C000E0FF22907F987416F090C000E0FF22907F987408F090C000E0FF22907F987409F090C000E0FF22907F98740AF090C000E0FF22907F98740BF090C000E0FFC0
:4013860022907F98740CF090C000E0FF22907F98740DF090C000E0FF22907F98740EF090C000E0FF22120FCF120D71120B4A220000000000000000000000000000000000C1
:4013C60000000000000000000000000000000000000000000000000000000000000000000000000000000000000000000000000000000000000000000000000000000000E7
:4014060000000000000000000000000000000000000000000000000000000000000000000000000000000000000000000000000000000000000000000000000000000000A6
:401446000000000000000000000000000000000000000000000000000000000000000000000000000000000000000000000000000000000000000000000000000000000066
:401486000000000000000000000000000000000000000000000000000000000000000000000000000000000000000000000000000000000000000000000000000000000026
:4014C60000000000000000000000000000000000000000000000000000000000000000000000000000000000000000000000000000000000000000000000000000000000E6
:4015060000000000000000000000000000000000000000000000000000000000000000000000000000000000000000000000000000000000000000000000000000000000A5
:401546000000000000000000000000000000000000000000000000000000000000000000000000000000000000000000000000000000000000000000000000000000000065
:401586000000000000000000000000000000000000000000000000000000000000000000000000000000000000000000000000000000000000000000000000000000000025
:4015C60000000000000000000000000000000000000000000000000000000000000000000000000000000000000000000000000000000000000000000000000000000000E5
:4016060000000000000000000000000000000000000000000000000000000000000000000000000000000000000000000000000000000000000000000000000000000000A4
:401646000000000000000000000000000000000000000000000000000000000000000000000000000000000000000000000000000000000000000000000000000000000064
:401686000000000000000000000000000000000000000000000000000000000000000000000000000000000000000000000000000000000000000000000000000000000024
:4016C60000000000000000000000000000000000000000000000000000000000000000000000000000000000000000000000000000000000000000000000000000000000E4
:4017060000000000000000000000000000000000000000000000000000000000000000000000000000000000000000000000000000000000000000000000000000000000A3
:401746000000000000000000000000000000000000000000000000000000000000000000000000000000000000000000000000000000000000000000000000000000000063
:401786000000000000000000000000000000000000000000000000000000000000000000000000000000000000000000000000000000000000000000000000000000000023
:4017C60000000000000000000000000000000000000000000000000000000000000000000000000000000000000000000000000000000000000000000000000000000000E3
:4018060000000000000000000000000000000000000000000000000000000000000000000000000000000000000000000000000000000000000000000000000000000000A2
:401846000000000000000000000000000000000000000000000000000000000000000000000000000000000000000000000000000000000000000000000000000000000062
:401886000000000000000000000000000000000000000000000000000000000000000000000000000000000000000000000000000000000000000000000000000000000022
:4018C6000000000000000000000000000000000000000000000000000000000000000000000000000000000000000000000000000000000000000000000012011001FF00BF
:401906000040CD06100100000102000209027400010100A032090400000EFF0000000705010240000007050202400000070503024000000705040240000007050502400076
:4019460000070506024000000705070240000007058102400001070582024000000705830240000107058402400001070585024000010705860240000107058702400001F4
:401986000403090448034B00650079007300700061006E002C002000610020006400690076006900730069006F006E0020006F006600200049006E006E006F005300790040
:4019C6007300200049006E0063002E0036034B00650079007300700061006E0020005500530042002000530065007200690061006C002000410064006100700074006500F9
:041A0600720000006A
:00000001FF
